S123A1003CBDA3D738BDA4C66D0026037EA184BDA5A5CEA904FFA9468601B7A944CEA944DA
S123A120BDD0067DA945263CB6A94885402645FEA94B2648FEA94DC6FF3AFFA8F9BCA8F29B
S123A140223A8610B7A944FEA8F0FFA948CEA944BDD0067DA9452614FEA8F908B6A901A73E
S123A160007EA184CEA855BDC0092072CEA866BDC009206ACEA878BDC0092062CEA773BDCE
S123A180C009205ACEA768BDC009BDA3E3BDA4E82447BDC021B6A8AF27EA84DF814926030C
S123A1A07EA1E1814426037EA23B815026037EA265815226037EA2C3815326037EA32C8129
S123A1C04826037EA3AB814E26037EA3B4815126037EA1DE863FBD7FE8BDC02120A67ED0DE
S123A1E003CEA8AFBDA4C6BDA460FEA8F98C00002605BDA6A42014FFA8F9BDA6A4FEA8F974
S123A200BCA8F6222DFFA8F6BDA6D0BDC021BDA3E37DA900270CCEA8F6BDA3F0CEA84ABD4E
S123A220C009BDA4E8240BBDA5D125DFCEA773BDC009BDC021BDC0217EA184CEA8AFBDA4CF
S123A240C6BDA4602519BDA6A4FEA8F98C0000270EBCA8F62209FFA8F6BDA6D0BDA663BDF6
S123A260C0217EA184CEA8AFBDA4C6BDA460240EFEA8F98C00002606CE0001FFA8F9BDA6EE
S123A280A4FEA8F9BCA8F62234FFA8F6BDA6D0BDC021B6A902B7A8F8BDA71FFEA8F46D0017
S123A2A0271BBD7FEBB1A9032713810D2708B6A902B7A8F820E28601B7A8F820DBBDC021AC
S123A2C07EA184CEA8AFBDA4C6BDA4602558BDA6A4FEA8F92750BCA8F6224BFFA8F6BDA669
S123A2E0D0BDC0218601B7A8F8BDA71FFEA8F609FFA8F67DA900270CCEA8F6BDA3F0CEA8BE
S123A3004ABDC009BDA3E3BDA4E8241ABDA6D0BDA5D1250CCEA773BDC009BDC0217EA18459
S123A320BDA6D0BDA663BDC0217EA184CEA88FBDC009BDA566BDA4E82459BDA594BDC02132
S123A340CEA904FFA946BDA6A48608B7A944CEA944BDD006FEA8F0FFA948FEA8F4BCA8F095
S123A360270E09BCA8F02708A600B1A901260109FFA94A8620B7A9448603B7A94CCEA944BB
S123A380BDD006CEA9446D01260FCEA896BDC0097EA184BDC0217EA184CEA8A0BDC009CEE8
S123A3A0A944BDA45CBDC0217EA184CEA788BDC0097EA1847DA900270F7FA900CEA851BD80
S123A3C0C009BDC0217EA1847CA900CEA84EBDC009BDC0217EA184FEA8F06F0008BCA8F25C
S123A3E026F839CEA8AF5F6F00085CC13F26F8397FA8FD8604B7A8FEEC00CEA4388D0B0813
S123A400087AA8FE26F7177EA4447FA8FFA100250D2204E1012507A3007CA8FF20EF36B688
S123A420A8FF260C7DA8FD26078620BD7FE820067CA8FDBDA4443239271003E80064000A3F
S123A44044444444840F8B30813923028B277E7FE8A600BDA440A600087EA4448DF38DF1CB
S123A4607FA8F97FA8FAA600272C81202728A60027228120271EBDA4AC241B81092E17BD01
S123A480A4987FA8FBB7A8FCFCA8F9F3A8FBFDA8F90820DA0C390D393637FCA8F905FDA8ED
S123A4A0F80505F3A8F8FDA8F9333239271680302B1281092F0C84DF81112B0881162E04E7
S123A4C080070D390C39A6002712812027030820F5A6002707812026030820F539A60027DE
S123A4E006BD7FE80820F6395FCEA8AFA6008100270BBD7FE8085CC13F220220EFBD7FEB18
S123A500B1A903275C817F27F422F28108270F81092724810D2743811F23E27EA54CC100C7
S123A52027DB095ABD7FE88620BD7FE88608BD7FE84FA7007EA4FDC13F27C28620BD7FE84A
S123A540A700085C17840726EE7EA4FDC13F27ADBD7FE8A700085C7EA4FDF7A8EF6F000DEB
S123A56039F7A8EF0C397FA8EFCEA904FFA8F9CEA8AFFFA8FBFEA8F9A600271208FFA8F9AD
S123A580FEA8FBA70008FFA8FB7CA8EF20E7FEA8FB6F00397FA8EFCEA8AFFFA8F9CEA9040C
S123A5A0FFA8FB20D0FFA8F9CEA904FFA8FBC664FEA8F9A60027148120271008FFA8F9FE20
S123A5C0A8FBA70008FFA8FB5A28E5FEA8FB6F0039FEA8F4A60081002705BDA62A2449CE1E
S123A5E0A8AFFFA8F9F6A8EF5D271BFEA8F9A60008FFA8F9FEA8F4A70008FFA8F408BCA8F7
S123A600F2271D5A20E2FEA8F4BCA8F22712B6A901A70008FFA8F4FEA8F608FFA8F60D394A
S123A620FEA8F4B6A901A7000C39FEA8F4A60008810026F9FFA8F9F6A8EF5C3AFFA8FBBC27
S123A640A8F2221DFEA8F9A60009FFA8F9FEA8FBA70009FFA8FBFEA8F9BCA8F40822E50D29
S123A660390C39FEA8F4FFA8F9A60081002734C601A60081002709B1A9012704085C20F183
S123A680FEA8F93AFFA8FBA6008100270BFEA8F9A70008FFA8F920E8FEA8FB096F00BCA86F
S123A6A0F926F839CE0001FFA8F6FEA8F0BCA8F22711FFA8F4A60081002708B1A90127043F
S123A6C00820EA39FCA8F6C30001FDA8F60820DDCE0001FFA8F9FEA8F0FFA8F4FEA8F68C65
S123A6E000012719FEA8F4BCA8F22711A6008100270BB1A901270708FFA8F420EA39FCA881
S123A700F9C30001FDA8F9B6A8F7B1A8FA260DB6A8F6B1A8F9260508FFA8F4390820C8FE64
S123A720A8F4BCA8F22240A6008100273A7DA8F82B0527337AA8F87DA900270CCEA8F6BDF6
S123A740A3F0CEA84ABDC009FEA8F4A60008FFA8F4B1A9012705BD7FE820EDFEA8F608FFDE
S123A760A8F6BDC02120B8393A3A2004537572653F20040D0A0A204F7574206F66206D658E
S123A7806D6F72790D0A0A040D0A204C696E6520656469746F722076312E320D0A20446160
S123A7A06E69656C20547566766573736F6E20323031372D323032320D0A0A20496E736553
S123A7C07274203C6C696E65206E756D6265723E0D0A2044656C657465203C6C696E6520F6
S123A7E06E756D6265723E0D0A205072696E74203C7374617274696E67206C696E65206E2C
S123A800756D6265723E0D0A205265706C616365203C6C696E65206E756D6265723E0D0AE6
S123A82020536176650D0A2048656C700D0A204E756D6265727320286F6E2F6F6666290DCD
S123A8400A20517569740D0A0A04203A20046F6E046F66660446696C65206E6F7420666F7E
S123A860756E640D0A0446696C652072656164206572726F720D0A04456E747279206973C3
S123A8802061206469726563746F72790D0A044E616D653A200453617665204F4B0D0A04E0
S112A8A053617665206661696C65642120240428
S107A8F001007DFFE3
S110A900010A141B756E7469746C656400A3
S115A944000000000000000000000000000000000000FD
S9030000FC
